:020000040000FA
:100000008A110A12AD2C0000F00003088301A3003E
:100010000A08A4000408A5000B1900000B18000032
:100020008B180000831203138A110A128C196020A6
:100030000C1B00008C1A00000C1A00000C190000A8
:100040008C1800000C1800000D1800008301250812
:10005000840024088A0023088300F00E700E090033
:1000C000831603171008110583128A110A120319E7
:1000D0008528AB008A110A122B19CF208A110A1227
:1000E0002B1889208A110A12AB19DB208A110A12F7
:1000F000AB1ABB208A110A12AB18C2208A110A124D
:100100002B1AAF208A110A126028831203138C1154
:100110000800AC01C4018316901190119011901148
:100120000830A100B830A2008830A000C030A6007E
:100130000830A40096019001831203138C118316DA
:100140000317063098003B309100FF3093000130D8
:10015000970083120130AD000313031708008316C4
:1001600011121012101111159514831203138C1112
:1001700003174414080083169012831203138C1182
:1001800003170800831690101208130592018312BA
:1001900003138C110317B000831203170800831692
:1001A00011111011101211169510831203138C11D6
:1001B0000317C40108008317831603171408A03E11
:1001C000840083120008A000840A0008A100840AA9
:1001D0000008A2008316031714089011831203135A
:1001E0008C110317C50020083C39B100243A8A114C
:1001F0000A12031928293108043A8A110A1203192C
:1002000008293108343A8A110A1203198A29080088
:1002100045088A110A12031D1D292E08213A8A1148
:100220000A12031D132983160830A1008830A0008C
:100230008A110A12831282290800083A8A110A12C6
:10024000031D232908004508103A03190800080077
:10025000450818398A110A12031D7B292E08063A0F
:100260008A110A12031D38298A110A127E247A295A
:100270002E08663A8A110A12031D44298A110A12AD
:100280007E248A110A127A292E08053A8A110A1246
:10029000031D50298A110A127B238A110A127A2916
:1002A0002E08033A8A110A12031D59298A110A12CB
:1002B0007A292E08013A8A110A12031D7729270884
:1002C000013A8A110A12031D6B298316191483122D
:1002D0008A110A127A292708023A8A110A12031D82
:1002E0007A2983161A1483128A110A127A298A1516
:1002F0000A12BD280800083A8A110A12031D812932
:100300000800080083160317A501C830A400831253
:10031000AE0108008317220884000008A300840AA5
:100320000008A400840A0008A500840A0008A600AA
:10033000840A0008A700840A0008A800840A0008AC
:10034000A900840A0008AA0083160830A100A400AE
:1003500083122308213A88300319C8308316A0007D
:1003600015128312AE0123088A110A120319E82913
:100370002308013A8A110A120319032A2308023AB0
:100380008A110A120319182A2308803A8A110A12BC
:100390000319242A2308813A8A110A120319362ADA
:1003A0002308823A8A110A120319482A230860395D
:1003B000203A8A150A120319002823086039403AA6
:1003C0008A110A12031D0C2B8A110A12AC2C080088
:1003D0002408013A8A110A120319872B2408053AC6
:1003E0008A110A1203196F2B2408093A8A110A127A
:1003F00003191C2C2408033A8A110A120319CB2B67
:100400008A110A120C2B2408013A8A110A120319C4
:10041000C82B24080B3A8A110A1203196B2C2408E2
:10042000033A8A110A1203190C2C8A110A120C2B96
:100430002408013A8A110A120319922B2408033A5C
:100440008A110A120319D62B2408083A8A110A12B3
:1004500003190F2C2408063A8A110A120319522A8A
:100460002408003A8A110A120319112B24080A3AA7
:100470008A110A1203194D2C2408003A8A110A1213
:100480000319202B2408063A8A110A120319522A4A
:100490002408003A8A110A1203194B2B8A110A12F6
:1004A0000C2B08002608223A8A150A120319542830
:1004B0002608213A8A150A120319A22802308A0056
:1004C000031026080339673E03188A0A82000C2BA2
:1004D0006B2A852AB52A0630AE000830B500E63012
:1004E000B2000830B3008A150A12E020B400AA084E
:1004F0008A110A12031D802A29022908031CB4004C
:10050000B40A8A110A127E2408000630AE000310D5
:10051000250D8A150A12CC20B2000310250D013ECC
:10052000CC20B3000230B2070318B30A8A150A12AE
:10053000E020B4000230B202031CB303AA088A11FF
:100540000A120319A62A8A110A12AE2A34082902AD
:100550008A110A120318AE2A2908B4000830B5001F
:10056000B40A8A110A127E2408006630AE002708F9
:100570008A110A12031DC62A2808031DC62A9230B2
:10058000B2000930B3008A110A12FD2A0930B30003
:100590009430B200BB018A150A125621B20A270212
:1005A0008A110A12031DDC2A8A150A125621280212
:1005B0008A110A120319E82AB20ABB0A98303202D9
:1005C0008A110A12031CCB2AAE018A110A120C2BC3
:1005D000063025028A110A12031CF22AAE018A1182
:1005E0000A120C2B250DB3003B088A150A125C2158
:1005F000B200B30A3B085C21B3008A150A125621E7
:10060000B40029022908031CB4000830B500B40A5C
:100610008A110A127E240800831603171814831205
:100620000800831626088400831283172D08800093
:10063000840A800183160230A500C830A400080097
:1006400083161708023A8A110A12031D2D2B8312F2
:1006500027088A110A12031D2D2B83161708033A47
:100660008A110A12031D0C2B83122708003C8A11E1
:100670000A12031C0C2B2708383E8400831700083D
:10068000F700831626088400770880000230A50052
:10069000C830A40008000F302705013A8A110A1259
:1006A0000319602B0F302705023A8A110A12031D25
:1006B0000C2B031083161A1803148A110A12642BC8
:1006C0000310831619180314260884008001800D76
:1006D000840A80010230A500C830A4000800250863
:1006E000AF008A110A12AF1B0C2B8A110A12822149
:1006F0000530AE000800AE01AC012F08831696004D
:100700008A110A120319862B023097000800250867
:10071000013A8A110A12031D0C2BAD108A110A121C
:100720008221080025088A110A12031D0C2B2608B5
:10073000031D0C2B831603301705023A8A110A1287
:10074000031DAD2B83120F302705031DAD2B831620
:1007500018108A110A128221080083160330170527
:10076000033A8A110A12031D0C2B83120F3027053E
:10077000023C8A110A12031C0C2B83170F30270529
:100780008316983E840000108A110A128221080004
:100790008A110A120C2B2508013A8A110A12031D2C
:1007A0000C2BAD148A110A128221080025088A1127
:1007B0000A12031D0C2B2608031D0C2B8316033075
:1007C0001705023A8A110A12031DF12B83120F300A
:1007D0002705031DF12B831618148A110A12822192
:1007E0000800831603301705033A8A110A12031D05
:1007F0000C2B83120F302705023C8A110A12031CAE
:100800000C2B83170F3027058316983E84000014A5
:100810008A110A12822108008A110A120C2B8316EF
:1008200026088400831283172C0880008316013069
:10083000A500C830A40008002508013C8A110A124E
:10084000031C0C2B2508AC008A110A1203192B2C4F
:100850008316033097008A110A1282218316031728
:10086000C830AA000830A9008830A8000830AD00C0
:10087000D030AE004830AC00D830B2000830B10003
:100880008830B0000830B500D830B6004830B40029
:100890000E3099000E309A00080083161708033AAC
:1008A0008A110A12031D0C2B83122708003C8A119F
:1008B0000A12031C0C2B2708383E840083170008FB
:1008C000F700831626088400770880000130A50011
:1008D000C830A40008008316170883120339033AAE
:1008E0008A110A12031D0C2B2708383E8400831737
:1008F000250880008A110A12822108008316031736
:1009000083172608840083120317B70137083502BE
:100910008A110A120319A02C8A110A12B40B932C03
:100920008A110A129F2C8A150A12E0208000B70A49
:10093000840A8A110A12B20F862CB30A862CAE01E1
:1009400037088316A5004030240640398838A400B3
:0A0950008A110A12080008000800CE
:06095A001E30F000F00B5E
:10096000AF2C8316031381178A150A12902383165E
:1009700003178A110A12640003301705033A031D96
:10098000BB2C831203138501860187010030F6001A
:100990008A110A12ED268A150A1283120313831391
:1009A00026308400083056228A110A12031CDB2CE0
:1009B0008A110A122026F4088A110A120319E82C57
:1009C000F4038312031303190516F6080319F42C14
:1009D0008A110A12D1278A110A120B258A110A12CA
:1009E000D8278A110A12BB27831203138A110A120D
:1009F000A6080319CB2C8A150A128313831203133A
:100A0000263084000830DA228A110A12031CFB2CDB
:100A10008A110A12CB2C8312031383132830AE00E1
:100A20003D088A110A12031D182DBE012730AE00A1
:100A300072088A110A12031DF72D3C088A110A1246
:100A4000031DF72D6030E5006C30EB000130EA004B
:100A5000F201B4010130E7003E08A6000310A60D24
:100A6000A60DA60DA60D4030E400A030E9003F0819
:100A7000AF003830A0000130E6000830BA00650849
:100A800084000008B200B3002E0884000301800037
:100A9000A2018A110A12582783160313C330860055
:100AA000EF308500FF3087008312031306116408BE
:100AB00084000008B0000608B100C039F50007083E
:100AC000C739E8000310F50CF50C750CE804E812C2
:100AD000B118E816E809B10922148A110A12582738
:100AE000A00A6808B0028A110A1203197B2D80003F
:100AF0008A110A12842D80000130311C0301B206D4
:100B00008A110A12321CA72D8A110A120C266508B6
:100B1000840066086609B30566083118B304330813
:100B200080006B0884006A086A18BC0AFF3CB405A0
:100B30006A083118B404340880000310EA0DEA088A
:100B40008A110A12031DA72DEB0A6A14B4010310BF
:100B5000E60DE40A0310B20C8A110A12BA0B482DF2
:100B600026086705031DAE0A0310E70D3830A007FD
:100B7000E50A8A110A12AF0B3B2DA030E90072087A
:100B80008A110A120319DF2D2E302E0203190800D4
:100B9000690883160313831384000008F30083128B
:100BA000031383132E08840073088000E90AAE0A39
:100BB000F2030430F40005128A110A12BF2D3C081A
:100BC000031908002E302E020319080083120313A4
:100BD00083136B0884000008F3002E088400730858
:100BE0008000EB0AAE0ABC038A110A12DF2D2830FE
:100BF000AE003D088A110A12031D012EBE012730E6
:100C0000AE003E08A6000310A60DA60DA60DA60D6B
:100C1000A6178A110A12BF2D6708A6042E088400A1
:100C2000000866048000F20A6908840068088316D8
:100C3000031383138000831203138313E90A08004C
:100C40008312031383130430BA0026308400000893
:100C50000A3C8A110A12031C3C2E0008B800840AC0
:100C60000408F1000008B6008A110A127B277108F7
:100C700084008A110A12E52E0008F73C8A110A1234
:100C80000318532E0008B800ED30B802840A040897
:100C9000F1000008B6008A110A127B27710884004F
:100CA0008A110A12E52E0008383C8A110A12031D27
:100CB0006D2E840A0408F1000008A2008A110A12AD
:100CC00042270830221C0A30B8008A110A12AF27C6
:100CD000710884008A110A12E52E0008393C8A1135
:100CE0000A12031D7A2E840A0008BD00BE008A1174
:100CF0000A12E52E00083A3C8A110A12031D862EBC
:100D0000840A0008BF008A110A12E52E0008FF3C81
:100D10008A110A12031D902E840A8A110A12E52EE6
:100D200000083B3C8A110A12031DA32E840A040802
:100D3000F1000008B8008A110A12AF277108840078
:100D40008A110A12E52E00083C3C8A110A12031D82
:100D5000B62E840A0408F1000008A2008A110A12C3
:100D60004227710884008A110A12E52E00083D3CD2
:100D70008A110A12031DCE2E840A0408F10000080D
:100D8000A2008A110A12ED268A110A121F270130C9
:100D9000F600710884008A110A12E52E0008A000EE
:100DA000840A0408F1000008B5000830BB00A20165
:100DB0000310B50CA20D8A110A125827A00A8A1135
:100DC0000A12BB0BD72E7108840083120313840A06
:100DD0008A110A12BA0B272E080083160313EF306C
:100DE0008500C3308600FF3087008316031302306E
:100DF0009F00831203139F171F13831603130C13F3
:100E000083120313861506150516F401F201BC01C1
:100E100083120313BD01BE010130BF00831203130F
:100E2000831340308400243083120313AF00030186
:100E30008000840A8A110A12AF0B182F412FA201D9
:100E40008A110A1242270430B000B1010130A20019
:100E50000830AF002F033107A0003830A0078A11F7
:100E60000A1258278A110A12AF0B2A2F4030B107F5
:100E70008A110A12B00B282F0A30B8008A110A1200
:100E8000AF2708000430B000A0010B30A0072D30C0
:100E9000AF008A110A125827A00A8A110A12AF0B52
:100EA000492F0830A0078A110A12B00B452F0800FD
:100EB000831203130C308600831603138701CF308F
:100EC0008500C03086008312031383132008A1001D
:100ED0003F39F500A10D03188616210D03180616DB
:100EE000C039750487008512F51985162218061475
:100EF000861186150800831203130630BB003608DE
:100F0000B700C039B2000A3EA0000130A2008A1129
:100F10000A1258273208A000A201B70CA20D8A11AC
:100F20000A125827A00A8A110A12BB0B8C2F043010
:100F3000BB003808B900A201B90CA20D8A110A122F
:100F40005827A00A8A110A12BB0B9B2FA2018A11F3
:100F50000A12582722148A110A1258270800FF3053
:100F600083120313AF00B6018A110A127B27B60A57
:100F7000AF0BB42F080083120313BD080319080038
:100F80003E08F500F503831603130C1383120313B5
:100F90009F121F129F1175189F15F5181F161F1409
:100FA000080083120313BD08031908001F15080069
:100FB000831203130615BD080319080083120313D7
:100FC0001F19DE2F831203130C13831203131E0841
:100FD00083120313A700BE03031D08003D08BE00D3
:020FE000080007
:101000008A150A122308213A031927288A150A1279
:101010002308223A0319C4288A150A122308233AFE
:101020000319C4288A150A122308A13A0319C428EF
:101030008A150A122308A23A0319C4288A150A122B
:101040002308A33A0319C4288A110A120C2B240876
:10105000013A8A150A120319C4282408023A8A158B
:101060000A120319C4282408033A8A150A1203191C
:10107000C4282408063A8A150A1203195428240899
:10108000093A8A150A120319C72824080A3A8A1548
:101090000A120319C42824080B3A8A150A120319E4
:1010A000C4288A110A120C2B831203170630AE00D3
:1010B0000830B5002608013A8A150A120319732868
:1010C0000310270D8A150A12D620B2000310270D2F
:1010D000013ED620B3008A150A12E020B400B20AFD
:1010E0008A150A1293282608023A8A150A12031949
:1010F0008C280310270D8A150A12D620B20003107F
:10110000270D013ED620B3008A150A12E020B40054
:10111000B20A8A150A1293282608033A8A110A127B
:1011200003190C2B08002A088A150A12031D9D2892
:101130002908340229080318B400B40A8A110A12D3
:101140007E2408000630AE000830B5000A30B20038
:101150000930B3008A150A12E020B400AA088A15E3
:101160000A12031DB72829022908031CB400B40A77
:101170008A110A127E24080008008A110A122E0819
:10118000063A03197E2408008A110A120C2B21301A
:10119000AE00831603170800F70008308A00D43029
:1011A000770703188A0A8200F8340834F7000830F9
:1011B0008A00DE30770703188A0A82002134093456
:1011C0008312031733088A00320882001234013474
:1011D0000034013400340034003408340034003466
:1011E000003400340034003402340134003401345B
:1011F0000934023429340034013401340434803495
:1012000032340934043400340034023403340034FA
:101210000034003409342134003401340034013402
:101220002234343400340734053481340334083430
:1012300000340A34073405340134033408340034EC
:101240000A3434340634A034FF3409340134A13470
:10125000013409340234A13400340634A134FF349B
:1012600009340334093404341534803425347F348C
:10127000353400344534FF3475340834953408343B
:101280008134023409340534093406341534803489
:1012900025347F34353400344534FF347534083414
:1012A0009534083491340234C034C03483120317A7
:1012B00033088A0032088200F7000310F70D8A1500
:1012C0000A126F21B600F70A8A150A126F21F70079
:1012D00077088A003608330703188A0A8200093023
:1012E0008A007630770703188A0A82007A34093434
:1012F000863409349234093498340934AC340934CE
:10130000C8340934D4340934DE340934923409340D
:10131000EE34093402340A3430340A343C340A34AA
:1013200046340A34063403340934043404340834AB
:1013300014340334493400344F340034433400341B
:101340006134003472340034643400345534003471
:1013500053340034423400341C3403344D340034EC
:10136000613400346E340034753400346534003434
:101370006C34003420340034563400346534003486
:101380006C340034653400347A3400342034003452
:101390000C34033456340034343400342E340034E6
:1013A00031340034303400340A34033443340034EC
:1013B000663400346734003431340034103403347C
:1013C0004E3400346F3400347434003468340034E4
:1013D000693400346E340034673400341434033418
:1013E0004D340034693400346334003472340034D2
:1013F0006F340034633400346834003469340034AA
:10140000703400342E3403345034003469340034E2
:10141000633400343134003436340034433400341F
:10142000373400343634003435340034203400345A
:101430005534003453340034423400342034003402
:10144000493400344F3400344334003461340034C0
:101450007234003464340034733400342034003483
:101460000C34033456340034343400342E34003415
:1014700031340034303400340A340334433400341B
:1014800066340034673400343134003410340334AB
:101490004E3400346F340034743400346834003413
:0C14A000693400346E34003467340034CA
:0414AC00030883129C
:1014B0000317C3000408BD00831603178A150A1218
:1014C000A81B922A290883120317C100C2008A159B
:1014D0000A120319822A831603172A088312031794
:1014E000BE0083173E0884000008F8003D08840011
:1014F000C31F831378088000BD0ABE0A8A150A122A
:10150000C10B712A831628084039403A8838A80050
:101510000830A90083124208F800430883007808C5
:101520000314080083120317430883000310080004
:10153000030883120317C3000408BD0083160317B2
:101540008A150A12B01BD42A310883120317C1006E
:10155000C2008A150A120319C42A83160317320817
:1015600083120317BE0083173E0884000008F800AA
:101570003D088400C31F831378088000BD0ABE0A9B
:101580008A150A12C10BB32A831630084039403A33
:101590008838B0000830B10083124208F8004308D0
:1015A000830078080314080083120317430883009C
:1015B00003100800F800030883120317C30078081B
:1015C0000F39C1000408BE004108831603178A15AD
:1015D0000A12AC1B112BAD008A150A120319052B38
:1015E0002E088312BD008317C31F83133E08840097
:1015F0000008F80083173D08840078088000BD0AC1
:10160000BE0A8A150A12C10BF32A83162C08403928
:10161000403A8838AC008312031743088300031450
:10162000080003100800F800030883120317C30022
:1016300078080F39C1000408BE004108831603175B
:101640008A150A12B41B4A2BB5008A150A1203190F
:101650003E2B36088312BD008317C31F83133E0839
:1016600084000008F80083173D0884007808800093
:10167000BD0ABE0A8A150A12C10B2C2B8316340828
:101680004039403A8838B400831203174308830076
:10169000031408000310080083170339983E8400E0
:1016A0000014080083170339983E840000100800D6
:1016B00083120317441C080083161011111595148A
:1016C000630000009510101211161011111108007E
:1016D00083120317AD1C0800831695101116101203
:1016E0001111101115158312BB018030BC008A1531
:1016F0000A12BB0B792BBC0B792B83161511080032
:101700008316031795118312BC01BB018A150A12B7
:10171000BB0F882BBC0F882B8A150A129023080058
:10172000831603179701013091009001083095004E
:101730008312AC010130AD00B801B901BA01FF302C
:10174000AE00831203138C1183168C150B178B17A5
:1017500008008316031795119514970103138C1134
:0217600008007F
:044000000034003454
:02400E00FA3F77
:00000001FF
